:1015D80090E600E0FFEF54E7FFEF4410FF90E600CD
:0315E800EFF022FF
:1010EB0041535345525400307825780047504946B8
:1010FB00545249473D257800475049464952513D86
:10110B0025780047504946544342333D25780047E4
:10111B00504946544342323D257800475049465486
:10112B004342313D25780047504946544342303DB8
:03113B0025780014
:1015960090E6087403F0438780D29ED29CD2997558
:0615A600B2017580002275
:101518008B6E8A6F89707BFF7A1079EB121097AB0C
:0B1528006EAA6FA97012109780FE22BF
:061097008B5D8A5E895F9B
:10109D00AB5DAA5EA95F8B608A618962121639AB5E
:1010AD0060AA61A962120BFEFFEF601E3099FDC2AE
:1010BD0099AB60AA61A962120BFEFF8F997401258D
:1010CD0062F562E43561F56180D53099FDC299759F
:0D10DD00990D3099FDC29975990A121639C6
:0110EA0022E3
:100003008F747B007A007934C003C002C0017BFF88
:100013007A1079F28B0B8A0C890D85740ED001D07E
:1000230002D00312044A7B007A007934121097221B
:1009D7007B007A007934C003C002C0017BFF7A1024
:1009E70079F78B0B8A0C890D85BB0ED001D002D00D
:1009F7000312044A7B007A0079341210977B007A3D
:100A0700007934C003C002C0017BFF7A1179038BE0
:100A17000B8A0C890D90E661E0FF8F0ED001D002A2
:100A2700D00312044A7B007A0079341210977B00B6
:100A37007A007934C003C002C0017BFF7A11790EB6
:100A47008B0B8A0C890D90E6CEE0FF8F0ED001D07C
:100A570002D00312044A7B007A0079341210977B84
:100A6700007A007934C003C002C0017BFF7A117994
:100A77001A8B0B8A0C890D90E6CFE0FF8F0ED00101
:100A8700D002D00312044A7B007A007934121097FF
:100A97007B007A007934C003C002C0017BFF7A1162
:100AA70079268B0B8A0C890D90E6D0E0FF8F0ED04C
:100AB70001D002D00312044A7B007A007934121065
:100AC700977B007A007934C003C002C0017BFF7AAC
:100AD7001179328B0B8A0C890D90E6D1E0FF8F0ECE
:100AE700D001D002D00312044A7B007A0079341275
:030AF70010972233
:04004F007580012295
:040DFC0075800022DC
:0416390063800122A7
:10153300536C6565700054445F53757370656E64D6
:0B154300000001020203030404050580
:10074A00752F00752E00752D00752C00C20DC20A7A
:10075A00C20CC20B1216417BFF7A0D7978AE02AF3A
:10076A00018E478F487BFF7A0D798AAE02AF018EE0
:10077A004F8F507BFF7A0D7994AE02AF018E458F71
:10078A00467BFF7A0D79B4AE02AF018E4D8F4E7B58
:10079A00FF7A0D79D4AE02AF018E518F527BFF7A68
:1007AA000D7978AE02AF01EE54E0FE7F00EF4E7095
:1007BA00030209397530007531807BFF7A0D79782B
:1007CA00AE02AF018E328F337BFF7A0D7978AE029B
:1007DA00AF017BFF7A0D79FAAC02AD01C3ED9FFF41
:1007EA00EC9EFEEF2402FFEE3400FEE4FCFD8F2BAC
:1007FA008E2A8D298C28752500752400752300758D
:10080A002200AF2BAE2AAD29AC28AB25AA24A923F6
:10081A00A822C3120C78503BAE24AF25AC30AD31C0
:10082A008D828C83E5822FF582E5833EF58374CD34
:10083A00F0AF25AE24AD23AC227B017A0079007893
:10084A0000EF2BF525EE3AF524ED39F523EC38F5D2
:10085A002280AF752500752400752300752200AF2C
:10086A002BAE2AAD29AC28AB25AA24A923A822C3DA
:10087A00120C785052AE24AF25AC32AD338D828C37
:10088A0083E5822FF582E5833EF583E0FFAC24AD54
:10089A0025AA30AB318B828A83E5822DF582E583E6
:1008AA003CF583EFF0AF25AE24AD23AC227B017A71
:1008BA000079007800EF2BF525EE3AF524ED39F5AD
:1008CA0023EC38F52280988530478531487BFF7ABA
:1008DA000D7978AE02AF01EF2480F527EE34FFF5EB
:1008EA0026C3E5509527F550E54F9526F54FC3E504
:1008FA004A9527F54AE5499526F549C3E54C9527D2
:10090A00F54CE54B9526F54BC3E5469527F546E5A7
:10091A00459526F545C3E54E9527F54EE54D9526B1
:10092A00F54DC3E5529527F552E5519526F551D275
:10093A00E843D82090E668E0FFEF4409FF90E668B4
:10094A00EFF090E65CE0FFEF443DFF90E65CEFF0ED
:10095A00D2AF90E680E0FFEF20E105D2091214271A
:10096A0090E680E0FFEF54F7FF90E680EFF0538EB9
:10097A00F8C20D300B05120056C20B300D497BFF31
:10098A007A157933121097121649503B7BFF7A1564
:10099A007939121097C20D1214D5200A2490E682D2
:1009AA00E0FFEF30E70990E682E0FFEF20E1E89010
:1009BA00E682E0FFEF30E60990E682E0FFEF20E012
:0C09CA00D612145612164D12164580A7C6
:0109D60022FE
:1000560090E6B9E0FFEF120C89018D00025F010303
:100066003603007B0601870801810901750A017BB9
:100076000B000003CC12004040030203DF90E6BBF6
:10008600E0FFEF120C89009F0100D702010F030069
:10009600BB0600F30700000164E547FF7E00EF544E
:1000A600FFFF90E6B3EFF0AF48EF54FFFF90E6B4E2
:1000B600EFF00203DFE54FFF7E00EF54FFFF90E60F
:1000C600B3EFF0AF50EF54FFFF90E6B4EFF002034A
:1000D600DFE549FF7E00EF54FFFF90E6B3EFF0AF98
:1000E6004AEF54FFFF90E6B4EFF00203DFE54BFF63
:1000F6007E00EF54FFFF90E6B3EFF0AF4CEF54FFF6
:10010600FF90E6B4EFF00203DF90E6BAE0FF1214C8
:1001160082AA06A9077B018B718A728973EA494B09
:10012600602BAB71AA72A973AE02AF01EEFF7E001F
:10013600EF54FFFF90E6B3EFF0AB71AA72A973AF6D
:1001460001EF54FFFF90E6B4EFF00203DF90E6A064
:10015600E0FFEF4401FF90E6A0EFF00203DF90E638
:10016600A0E0FFEF4401FF90E6A0EFF00203DF12EC
:1001760015FE0203DF1216300203DF1200460203E9
:10018600DF1215EB0203DF12165140030203DF9064
:10019600E6B8E0FFEF120C8901AB8001D48101ECD7
:1001A600820000024EA20AE433FFEF25E0FFA20C14
:1001B600E433FEEF4EFF90E740EFF090E741E4F0C6
:1001C60090E68AE4F090E68B7402F00203DF90E793
:1001D60040E4F090E741E4F090E68AE4F090E68BA4
:1001E6007402F00203DF90E6BCE0FFEF547EFF7E70
:1001F6000090E6BCE0FDEDD3948040067C007D01D6
:1002060080047C007D00EC4EFEED4FFF74442FF51C
:100216008274153EF583E493FFEF3395E0FEEF24F9
:10022600A1FFEE34E6FE8F828E83E0FFEF5401FFDE
:1002360090E740EFF090E741E4F090E68AE4F09032
:10024600E68B7402F00203DF90E6A0E0FFEF4401C4
:10025600FF90E6A0EFF00203DF12165340030203FD
:10026600DF90E6B8E0FFEF120C89027A00029902ED
:10027600000003DF90E6BAE0FFEFB40105C20A0210
:1002860003DF90E6A0E0FFEF4401FF90E6A0EFF069
:100296000203DF90E6BAE0FFEF600302032290E676
:1002A600BCE0FFEF547EFF7E0090E6BCE0FDEDD3A0
:1002B600948040067C007D0180047C007D00EC4E2D
:1002C600FEED4FFF74442FF58274153EF583E493DB
:1002D600FFEF3395E0FEEF24A1FFEE34E6FE8F82BA
:1002E6008E83E0FFEF54FEFFEFF090E6BCE0FFEFF9
:1002F6005480FFEF131313541FFF90E6BCE0FEEE8D
:10030600540FFEEF2EFF90E683EFF090E683E0FFBA
:10031600EF4420FF90E683EFF00203DF90E6A0E0D3
:10032600FFEF4401FF90E6A0EFF00203DF0203DFD8
:1003360012165540030203DF90E6B8E0FFEF120CF9
:1003460089035100037C02000003DF90E6BAE0FF58
:10035600EFB40105D20A0203DF90E6BAE0FFEFB47C
:1003660002048075807390E6A0E0FFEF4401FF90E1
:10037600E6A0EFF0806390E6BCE0FFEF547EFF7EE0
:100386000090E6BCE0FDEDD3948040067C007D0144
:1003960080047C007D00EC4EFEED4FFF74442FF58B
:1003A6008274153EF583E493FFEF3395E0FEEF2468
:1003B600A1FFEE34E6FE8F828E83E0FFEF4401FF5D
:1003C600EFF080158013121657500E90E6A0E0FF4E
:1003D600EF4401FF90E6A0EFF090E6A0E0FFEF44C7
:0703E60080FF90E6A0EFF09C
:0103ED0022ED
:0300330002163D75
:04163D0053D8EF325D
:1014560090E682E030E004E020E60B90E682E030A1
:10146600E119E030E71590E680E04401F07F147E54
:0C1476000012135790E680E054FEF022B4
:1014D50090E682E044C0F090E681F0438701000089
:0414E50000000022E1
:1014270030090990E680E0440AF0800790E680E002
:101437004408F07FDC7E0512135790E65D74FFF0D9
:0F14470090E65FF05391EF90E680E054F7F022CB
:02148200A907B8
:10148400AE51AF528F828E83A3E064037017AD0117
:1014940019ED7001228F828E83E07C002FFDEC3EDB
:0914A400FEAF0580DF7E007F0031
:0114AD00221C
:101357008E1C8F1D90E600E054187012E51D2401C5
:10136700FFE4351CC313F51CEF13F51D801590E63C
:1013770000E05418FFBF100BE51D25E0F51DE51C27
:1013870033F51CE51D151DAE1C7002151C4E6005BE
:061397001214E980EE22B1
:1014E9007400F58690FDA57C05A3E582458370F916
:0114F90022D0
:03004300020E00AA
:03005300020E009A
:100E000002154E000215C2000215AC000215660064
:100E10000212C700021191000200420002165D009A
:100E200002165E0002165F000216600002122F001A
:100E300002127B00021661000216620002166300B5
:100E40000216640002165D000216650002166600B6
:100E500002166700021668000216690002166A0090
:100E600002166B0002165D0002165D0002165D00A0
:100E700002166C0002166D0002166E0002166F005C
:100E8000021670000216710002167200021673003C
:100E9000021674000216750002167600021677001C
:100EA0000213E300021678000216790002167A0097
:080EB00002167B0002167C0013
:0611E3008B538A5489556C
:1011E900755B00755C00C3E55C955AE55B955950E4
:1011F90034AB53AA54A955120BFEFFAB56AA57A9F3
:1012090058EF120C4474012558F558E43557F55731
:1012190074012555F555E43554F554055CE55C70C4
:0512290002055B80C11D
:01122E00229D
:08103B008B638A6489658D66F0
:10104300E566540FF567E566C4540FF568E567C3B5
:10105300940A500874302567F5678006743725674E
:10106300F567E568C3940A500874302568F568800D
:101073000674372568F568AB63AA64A965E5681249
:101083000C44AB63AA64A965758201758300E567A7
:03109300120C56E6
:011096002237
:100D780012010002FFFFFF4025098138000001022F
:100D880000010A060002FFFFFF40010009022000DF
:100D980001010080320904000002FFFFFF0007057F
:100DA8000102000200070582020002000902200079
:100DB80001010080320904000002FFFFFF0007055F
:100DC80001024000000705810240000004030904F5
:100DD8001603530061006C00650061006500200087
:100DE8004C004C0043000C034C006F006700690086
:040DF8006300000094
:0416410012113E2222
:0416450012167D22DA
:0416490012165922FA
:04164D0012165B22F4
:02004000D322C9
:0900460090E6BAE0FF8F1FD322FF
:1015EB0090E740E51FF090E68AE4F090E68B7401FB
:0315FB00F0D32208
:0916300090E6BAE0FF8F1ED32200
:1015FE0090E740E51EF090E68AE4F090E68B7401E9
:03160E00F0D322F4
:02165100D322A2
:02165300D322A0
:02165500D3229E
:02165700D3229C
:10154E00C0E0C083C082D20B5391EF90E65D740170
:08155E00F0D082D083D0E0320E
:1015AC00C0E0C083C0825391EF90E65D7404F0D02C
:0615BC0082D083D0E03272
:1015C200C0E0C083C0825391EF90E65D7402F0D018
:0615D20082D083D0E0325C
:1012C700C0E0C083C082C0D075D000C006C007850B
:1012D7004D49854E4AAE49AF4A8F828E83A3740229
:1012E700F085454B85464CAE4BAF4C8F828E83A322
:1012F7007407F05391EF90E65D7410F0D007D006B5
:09130700D0D0D082D083D0E032B6
:10156600C0E0C083C082D20D5391EF90E65D74084F
:08157600F0D082D083D0E032F6
:10119100C0E0C083C082C0D075D000C006C0079037
:1011A100E680E0FFEF30E72485454985464AAE49B0
:1011B100AF4A8F828E83A37402F0854D4B854E4CCE
:1011C100AE4BAF4C8F828E83A37407F05391EF9097
:1011D100E65D7420F0D007D006D0D0D082D083D085
:0211E100E032FA
:01004200328B
:01165D00325A
:01165E003259
:01165F003258
:011660003257
:10122F00C0E0C0F0C083C082C0D075D000C000C085
:10123F0001C002C003C004C005C006C0075391EF30
:10124F0090E65FE0FFEF4408FF90E65FEFF01213C8
:10125F009DD007D006D005D004D003D002D001D046
:0C126F0000D0D0D082D083D0F0D0E0328C
:10127B00C0E0C0F0C083C082C0D075D000C000C039
:10128B0001C002C003C004C005C006C0075391EFE4
:10129B0090E65FE0FFEF4410FF90E65FEFF0120087
:1012AB0036D007D006D005D004D003D002D001D061
:0C12BB0000D0D0D082D083D0F0D0E03240
:011661003256
:011662003255
:011663003254
:011664003253
:011665003252
:011666003251
:011667003250
:01166800324F
:01166900324E
:01166A00324D
:01166B00324C
:01166C00324B
:01166D00324A
:01166E003249
:01166F003248
:011670003247
:011671003246
:011672003245
:011673003244
:011674003243
:011675003242
:011676003241
:011677003240
:1013E300C0E0C0F0C083C082C0D075D000C000C0D0
:1013F30001C002C003C004C005C006C0075391BFAB
:1014030090E6517401F0121611D007D006D005D022
:1014130004D003D002D001D000D0D0D082D083D06A
:04142300F0D0E032F3
:01167800323F
:01167900323E
:01167A00323D
:01167B00323C
:01167C00323B
:100FC7004F6E457032496E004F766572666C6F776B
:100FD7000067706966207761736E27742072656198
:100FE70064790045503220494E20776173206E6F37
:100FF7007420636F6D706C65746C7920656D7074A7
:1010070079207768656E20617474656D7074696E98
:101017006720746F20737461727420746865206729
:10102700706966005374617274202825642900531F
:04103700746F700062
:020CBF00C10E64
:10113E001215D812159612004FD20A00000090E632
:10114E000B7403F00000000000001214FA121310CA
:10115E00120AFA90E668E0FFEF4403FF90E668EFAC
:10116E00F00000005391BF00000090E6517401F0B2
:10117E0000000090E6507401F000000043E8040007
:03118E000000223C
:01167D00224A
:10139D007B017AE779808B698A6A896BAB69AA6A66
:0D13AD00A96B120BFEFF8F6CE56CB40117ED
:1013BA00AB69AA6AA96B758201758300120C17FFC3
:0713CA008F6DAF6D120F449F
:1013D100E56CB4020312157E00000090E68D7440A6
:0113E100F01B
:0113E20022E8
:0A0036007BFF7A0F79C712109722A2
:1016110012157E7BFF7A0F79CF1210971209D7220C
:02165900D3229A
:02165B00C322A8
:1014FA0090E61074A0F090E65EE0FFEF4408FF90DB
:0E150A00E65EEFF000000090E68D7440F022E7
:1013100090E61274E0F000000090E6047480F000A3
:10132000000090E6047402F000000090E604E4F08F
:1013300000000090E6187408F000000090E6D274F7
:1013400002F000000090E6207402F000000090E639
:0713500021E4F0000000227F
:100F44008F75121310AF7512162180147BFF7A0F60
:100F540079D812151880097BFF7A0F79EA121518CF
:100F640000000090E6CE74FFF000000090E6CF741D
:100F7400FFF000000090E6D074FFF000000090E65F
:100F8400D174FFF000000075BB04AF757E008E4382
:100F94008F447B007A007934C003C002C0017BFF18
:100FA4007A10792B8B0B8A0C890D85430E85440F9F
:100FB400D001D002D00312044A7B007A00793412A3
:030FC40010972261
:0F1621008F76759DE4759E0090E67CE576F0224D
:10157E0090E6D2E4F000000090E6D37401F07BFF19
:08158E007A1079361210972241
:100CC100608017700138010101010107020900006C
:100CD10000000000000000000000000000360000DD
:100CE1000000003F010101010101010700000000B6
:100CF10000000000000000000000000000000000F3
:100D01000000003F01010101010101070000000095
:100D110000000000000000000000000000000000D2
:100D21000000003F04010101010101070000000072
:100D310000000000000000000000000000000000B2
:100D41000000003F602417F70000000000000000D1
:100D51000000000000000000000000000000000092
:100D61000000000000000000000000004717F0E054
:060D7100000000CEC400EA
:100AFA0090E60174CEF090E6F574FFF09017F0E0FE
:100B0A00FF90E6F3EFF09017F1E0FF90E6C3EFF005
:100B1A009017F2E0FF90E6C1EFF09017F3E0FF9034
:100B2A00E6C2EFF09017F5E0FF90E6C0EFF09017FD
:100B3A00F6E0FF90E6F4EFF075AF077B017A1779DC
:100B4A0070AE02AF01EEFF7E00EF54FFF59A7B0113
:100B5A007A177970AF01EF54FFF59B759DE4759E86
:100B6A0000757700E577C39480500E90E67BE0FF2E
:100B7A0090E67CEFF0057780EB90E67174FFF075F4
:100B8A00B4FF90E672E0FFEF4480FF90E672EFF068
:100B9A0043B68000000090E6C4E4F000000090E64E
:100BAA00C5E4F09017F7E0FF90E6C6EFF09017F86B
:100BBA00E0FF90E6C7EFF09017F9E0FF90E6C8EF84
:100BCA00F09017FAE0FF90E6C9EFF09017FBE0FF0C
:100BDA0090E6CAEFF09017FCE0FF90E6CBEFF090BA
:100BEA0017FDE0FF90E6CCEFF09017FEE0FF90E6ED
:030BFA00CDEFF04C
:010BFD0022D5
:03000000020EB835
:0C0EB800787FE4F6D8FD758177020EFF0C
:100BFE00BB010689828A83E0225002E722BBFE02F5
:090C0E00E32289828A83E4932227
:100C1700BB010CE58229F582E5833AF583E0225092
:100C270006E92582F8E622BBFE06E92582F8E222DC
:0D0C3700E58229F582E5833AF583E49322F6
:100C4400BB010689828A83F0225002F722BBFE018F
:020C5400F32289
:100C5600F8BB010DE58229F582E5833AF583E8F0D4
:100C6600225006E92582C8F622BBFE05E92582C880
:020C7600F22268
:100C7800EB9FF5F0EA9E42F0E99D42F0E89C45F0D2
:010C88002249
:100C8900D083D082F8E4937012740193700DA3A3FA
:100C990093F8740193F5828883E47374029368600E
:060CA900EFA3A3A380DF0E
:1003EE00E517240BF8E60517227808300702780B7C
:1003FE00E475F001120CAF020BFE2000EB7F2ED243
:10040E00008018EF540F2490D43440D4FF30040BE6
:10041E00EF24BFB41A0050032461FFE518600215E3
:10042E0018051BE51B7002051A30070D7808E475D8
:10043E00F001120CAFEF020C440214AE7403D2079B
:10044E008003E4C207F5178B088A09890AE4F518B8
:10045E00F51AF51BE51860077F2012042980F57543
:10046E0019FFC201C200C202C203C205C206C208FF
:10047E001203F7FF700D3007057F0012043AAF1B11
:10048E00AE1A22B4255FC2D5C2041203F7FF24D0E0
:10049E00B40A00501A75F00A781830D50508B6FF60
:1004AE000106C6A426F620D5047002D20380D924F4
:1004BE00CFB41A00EF5004C2E5D20402063AD201BC
:1004CE0080C6D20080C0D20280BCD2D580BAD205FE
:1004DE0080B47F201204292002077401B518004051
:1004EE00F11203EEFF120429020462D208D2068032
:1004FE00951203EEFB1203EEFA1203EEF94A4B705D
:10050E0006790B7A077BFF20022EE518602A7E0003
:10051E008E82758300120C1760060EEE651970F050
:10052E00C2D5EBC0E0EAC0E0E9C0E0EE120681D031
:10053E00E0F9D0E0FAD0E0FB120BFEFF60AAEBC0B0
:10054E00E0EAC0E0E9C0E0120429D0E02401F9D0CD
:10055E00E03400FAD0E0FBE5190460DCD519D9804F
:10056E00877BFF7A06797DD202809C791080027992
:10057E0008C206C2088008D2D5790A8004790AC258
:10058E00D5E519047002F519E4FAFDFEFF1203EE2B
:10059E00FC7B082001131203EEFD7B1030000A12C3
:1005AE0003EEFE1203EEFF7B20EC3382D592D55084
:1005BE0013C3E43000069FFFE49EFEE42001039D7A
:1005CE00FDE49CFCE4CBF8C201EC700CCFCECDCC9C
:1005DE00E824F8F870F38017C3EF33FFEE33FEED27
:1005EE0033FDEC33FCEB33FB994002FB0FD8E9EB08
:1005FE00300105F8D0E0C448B201C0E00AEC4D4E1F
:10060E004F78207B0070C2EAB5190040BCC0E012E2
:10061E000683D0F0D0E0200104C4C0E0C4B201C013
:10062E00F0120412D0F0D5F0EB020462120C890421
:10063E00FF5305795804D04C04CC42057D4F0585F7
:0F064E004405854904E543058B55056F46056F47
:10065D0045056F47072B5004D42D04D82E04FB2BD2
:10066D0004DC2304F92007142A049448000004F341
:10067D003F3F3F00790AA2D5200314300509B91078
:10068D00020404B9080104A2D52006025001042079
:10069D0002689202B518005034C0E07F2030031973
:1006AD007F30A20272067205500F1206DAC202C224
:1006BD0006C205C2087F30800F300503E9C0E01285
:1006CD000429300503D0E0F9D0E0B518CC3005177A
:1006DD007F30B9100C1204297F583004077F7880C1
:1006ED0003B908031204293002057F2D0204297F66
:1006FD00202008F87F2B2006F322920280CF286E4F
:10070D00756C6C2900D2011203EE3001F8C201782C
:10071D001830D50108F60204942D504349581203A0
:10072D00EE2403B405004001E49007269312041A49
:0D073D00743A12041AD203751804020579EB
:100EC40002074AE493A3F8E493A34003F68001F2F3
:100ED40008DFF48029E493A3F85407240CC8C3332F
:100EE400C4540F4420C8834004F456800146F6DFFE
:100EF400E4800B0102040810204080900CBFE47EC3
:100F0400019360BCA3FF543F30E509541FFEE493F2
:100F1400A360010ECF54C025E060A840B8E493A3B9
:100F2400FAE493A3F8E493A3C8C582C8CAC583CAE4
:100F3400F0A3C8C582C8CAC583CADFE9DEE780BE9C
:010D7700007B
:100CAF00FAE6FB0808E6F925F0F618E6CA3AF62246
:1014AE00EFB40A07740D1214B9740A309811A89982
:1014BE00B8130CC2983098FDA899C298B811F6309E
:0714CE0099FDC299F5992276
:00000001FF
